:100000000C941E060C943B280C9468280C9446060D
:100010000C9446060C9446060C9446060C94460630
:100020000C9446060C9446060C9432130C94460627
:100030000C9446060C9446060C9446060C94460610
:100040000C9495280C9446060C94832C0C94C62C86
:100050000C9446060C9446060C9446060C944606F0
:100060000C9446060C944606BB181D19FC18FF1884
:100070000219051908190B190E191D1917194F1A0C
:10008000511A511A4F1A511A511A511A511A511A1A
:10009000511A511A511A511A511A511A511A511A08
:1000A000D519511A511A511A511A511A4619511A81
:1000B000511A511A511A511A511A511A511A511AE8
:1000C000511A511A511A511A511A511AE119E119BA
:1000D000E119E119E119E119E119E119E119511ADF
:1000E000511A511A511A511A511A4619E019E019A8
:1000F000E019E019511AEE19F419FA19001A061A42
:100100000C1A121A181A221A2C1A361A401A87199F
:100110004919511A511A511A511AD519511A511A0D
:10012000511A511A511A511A511A511ADF19DF195D
:10013000DF19DF19511AEE19F419FA19001A061A03
:100140000C1A121A181A221A2C1A361A401A87195F
:100150004919511A511A511A511AD519841A841A67
:10016000841A841A841A841A841A841A841A841A9F
:10017000841A841A841A9B1B9B1B9B1B9B1B9B1B17
:100180009B1BC91AD31ADD1AE71A451B4F1B5E1BAE
:100190006F1BF71C0C1D181D211D301D551D5E1DEC
:1001A000A71D701DBA20C020C620CD20DB20FD2059
:1001B0001B21456E746572206D656E752E2E2E00A6
:1001C000546F67676C6564206D6963726F50504D42
:1001D00000546F67676C656420696E76657274653C
:1001E000642050504D2100546F67676C6564205443
:1001F00058206D7574696E672100546F67676C6570
:10020000642074656C656D65747279210050726F3D
:10021000746F636F6C206572726F72207769746897
:100220002052580054696D656F7574207768656E4B
:1002300020636F6E6E656374696E6720746F205201
:100240005800507265737320616E79206B65792058
:10025000746F2063616E63656C00436F6E6E6563DF
:1002600074696E6720746F2052582C20706F776508
:100270007220757020746865205258202877697440
:10028000682062696E6420706C7567206966206EF4
:100290006F74207573696E6720616C776179732064
:1002A00062696E642900546F67676C656420276912
:1002B0006D6D656469617465206F75747075742700
:1002C00000546F67676C65642027736C61766520E6
:1002D0006D6F64652700546F67676C6564202761E4
:1002E0006C776179732062696E642700546F676769
:1002F0006C65642050504D206368616E6E656C20A3
:100300006C696D69740053657420525353492069B8
:100310006E6A656374696F6E206368616E6E656C8A
:100320002028303D3D64697361626C652900536526
:10033000742050504D206D696E696D756D20737914
:100340006E630053657420626561636F6E20696E31
:1003500074657276616C0053657420626561636FC9
:100360006E2064656C617900536574206265616319
:100370006F6E206672657175656E637920696E2097
:10038000487A3A20303D64697361626C652C205074
:10039000783D504D52206368616E6E656C20782CFC
:1003A0002046783D465253206368616E6E656C202E
:1003B00078005365742050574D2073746F7020641B
:1003C000656C61792028302064697361626C6564B2
:1003D0002C20312D323535203D3D20302E317320FB
:1003E0002D2035306D696E29005365742050504DB5
:1003F0002073746F702064656C61792028302064EC
:10040000697361626C65642C20312D323535203D75
:100410003D20302E3173202D2035306D696E29003E
:10042000536574206661696C736166652064656CF0
:1004300061792028302064697361626C65642C20C6
:10044000312D323535203D3D20302E3173202D2089
:1004500035306D696E29002A2A2A2A2A2A2A2A2A50
:100460002A2A2A2A2A2A2A2A2A2A2A2A2A2A2A2AEC
:100470002A2A2A2A0052582041636B6564202D20C5
:1004800072657665727420737563636573736675E0
:100490006C21002A2A2A2A2A2A2A2A2A2A2A2A2AAD
:1004A0002A2A2A2A2A2A2A2A2A2A2A2A2A2A2A2AAC
:1004B000002A2A2A2A2A2A2A2A2A2A2A2A2A2A2AC6
:1004C0002A2A2A2A2A2A2A2A2A2A2A2A2A2A00528E
:1004D000582041636B6564202D20757064617465DC
:1004E000207375636365737366756C21002A2A2A0D
:1004F0002A2A2A2A2A2A2A2A2A2A2A2A2A2A2A2A5C
:100500002A2A2A2A2A2A2A2A2A2A0056616C696457
:100510002063686F69636573206172653A205B319F
:100520005D2D5B31365D20286368616E6E656C20E1
:10053000312D31362900536574206F7574707574D0
:1005400020666F7220706F727420005B585D2061AE
:10055000626F7274206368616E67657320616E6498
:10056000206578697420525820636F6E6669670051
:100570005B535D20736176652073657474696E6783
:100580007320746F205258005B525D20726576654F
:1005900072742052582073657474696E6773207486
:1005A0006F2064656661756C747300557365206EA9
:1005B000756D62657273205B312D445D20746F2010
:1005C0006564697420706F727473205B452D515D92
:1005D00020666F722073657474696E677300202DD6
:1005E00020726563656976657220636F6E66696700
:1005F000757261746F722C20727820737720000AF4
:100600000A6F70656E4C52536E67200053657420FC
:1006100073657269616C2062617564726174653AB8
:10062000200056616C69642063686F696365733A82
:100630002031202D20342B34202F2032202D203823
:10064000202F2033202D20382B34202F2034202D14
:10065000203132202F2035202D2031322B34202FF5
:100660002036202D20313600536574204368616E9A
:100670006E656C20636F6E6669673A20005365741F
:100680002044617461726174652028302D32293AEA
:10069000200053657420486F70206368616E6E653A
:1006A0006C7320286D61782032342C207365706162
:1006B000726174656420627920636F6D6D61732966
:1006C0002076616C69642076616C75657320312DCC
:1006D0003235353A2000536574206368616E6E656B
:1006E0006C2073706163696E6720287831306B48C5
:1006F0007A293A200053657420524620706F77653E
:10070000722028302D37293A200053657420524634
:10071000206D6167696320286865782920652E67E8
:100720002E20307844454144463030443A2000532E
:1007300065742062617365206672657175656E63AC
:10074000792028696E20487A293A20005B5A5D207A
:10075000656E746572207265636569766572206383
:100760006F6E66696775726174696F6E2075746902
:100770006C79005B465D20646973706C61792061FF
:10078000637475616C206672657175656E63696509
:10079000732075736564005B525D2063616C6375E3
:1007A0006C6174652072616E646F6D206B65792079
:1007B000616E6420686F70206C697374005B495DC2
:1007C000207265696E697469616C697A6520736508
:1007D0007474696E677320746F20736B65746368DB
:1007E0002064656661756C7473005B585D2072658A
:1007F00076657274206368616E67657320616E64EC
:100800002065786974206D656E75005B535D20739B
:100810006176652073657474696E677320746F20E8
:10082000454550524F4D20616E64206578697420B3
:100830006D656E7500557365206E756D62657273BA
:10084000205B302D395D20746F20656469742070E1
:100850006172616D657465727300202D2053797328
:1008600074656D20636F6E66696775726174696F18
:100870006E000A0A6F70656E4C52536E672000510D
:1008800029204F7574707574206265666F726520DB
:100890006C696E6B20283D465329203A2000502970
:1008A00020536C617665206D6F64652028657870D3
:1008B0006572696D656E74616C293A20004F29205C
:1008C00054696D65642042494E44206174207374FC
:1008D000617274757020203A20004E292050504DCE
:1008E000206F7574707574206C696D69746564200F
:1008F000202020203A200044495341424C454400E6
:100900004D292050504D205253534920746F20637D
:1009100068616E6E656C202020203A20004C2920F2
:1009200050504D206D696E696D756D2073796E63E1
:10093000202875732920203A200044495341424C15
:100940004544004B29204661696C736166652062ED
:100950006561636F6E20696E74762E2028312D32AA
:10096000353573293A20004A29204661696C736144
:10097000666520626561636F6E2064656C617920D5
:1009800028302D323535203D3E20313073202D204A
:100990003135306D696E293A200049292046616958
:1009A0006C7361666520626561636F6E206672714B
:1009B0002E203A200048292050574D2073746F7024
:1009C0002064656C6179202020202020203A2000BE
:1009D00047292050504D2073746F702064656C61FE
:1009E00079202020202020203A200046292046611E
:1009F000696C736166652064656C617920202020D4
:100A00002020203A200050574D206368616E6E65AB
:100A10006C200066756E6374696F6E3A2000292041
:100A2000706F72742000506F776572546F776572C3
:100A300000445446205548462033322D62697420C4
:100A400031306368004F70656E4C52536E67525878
:100A5000206D696E6920342F36636800466C7974A6
:100A6000726F6E2F4F72616E6765525820554846FF
:100A70002038636800525820747970653A20004429
:100A8000697361626C656400487A00203D3D200016
:100A900043616C63756C61746564207061636B6540
:100AA0007420696E74657276616C3A200042292068
:100AB0004D6963726F202868616C66292050504D23
:100AC000202020203A00412920496E766572746505
:100AD000642050504D20696E20202020203A0030A4
:100AE00029204D7574652062757A7A657220286DAB
:100AF0006F73746C79293A003929205365726961E2
:100B00006C2062617564726174653A00736D617224
:100B100074506F7274004672536B79005472616E38
:100B200073706172656E740044697361626C6564B0
:100B30000038292054656C656D657472793A2020FF
:100B40002020202020003729204368616E6E656CCC
:100B500020636F6E6669673A202000362920446161
:100B60007461726174652028302D32293A2020206A
:100B700000352920486F70206368616E6E656C7364
:100B80003A2020202020003429204368616E6E65C1
:100B90006C2073706163696E673A202000332920EE
:100BA000524620706F7765722028302D37293A2001
:100BB0002020003229205246206D616769633A2067
:100BC0002020202020202020003129204261736530
:100BD000206672657175656E63793A202020000089
:100BE00000000700020100000304060000000000EE
:100BF00000000001020408102040800102040810D7
:100C00002001020408102004040404040404040263
:100C10000202020202030303030303000000002395
:100C2000002600290000000000250028002B0000FD
:100C3000000000240027002A0000B42D11241FBE4C
:100C4000CFEFD8E0DEBFCDBF13E0A0E0B1E0E6E734
:100C5000F1E602C005900D92A83CB107D9F716E065
:100C6000A8ECB3E001C01D92AE38B107E1F71CE07B
:100C7000CCE3DCE004C02297FE010E94BD2ECA3303
:100C8000D107C9F70E94F02D0C94B9300C940000E4
:100C900080917305813019F482E08093730580910F
:100CA0007305833019F484E0809373050895A89543
:100CB0000895DC01ED91FC910190F081E02D099502
:100CC00008952091740530917505382748E0C901D1
:100CD000880F991F37FF06C09C0151E2252750E17C
:100CE000352701C09C01415091F730937505209341
:100CF0007405089588E38093760580E092ECA1E086
:100D0000B0E08093770590937805A0937905B09330
:100D10007A0587E08093830580EC9AECA9E8B6E336
:100D200080937B0590937C05A0937D05B0937E0511
:100D300085E0809384058DEE9EEFADEABEED809355
:100D40007F0590938005A0938105B0938205E5E827
:100D5000F5E080E090E0863028F4DC01AE54BC4F32
:100D60002C9101C020E0219301968831910599F7DB
:100D700082E080939D058AE080939E05089580EC33
:100D800097EFAAEBB7E38093BB059093BC05A093C4
:100D9000BD05B093BE0580E090E0A0E0B0E5809393
:100DA000BF059093C005A093C105B093C205E3ECC5
:100DB000F5E080E081938F5F8031E1F70895A0E056
:100DC000B0E0E5EEF6E00C94862ED82F0E94EB28DA
:100DD0006115710581059105C9F30E94292F1092B3
:100DE0007F05109280051092810510928205C4E063
:100DF000812C912C54018A94C0907F05D09080055D
:100E0000E0908105F0908205FE2CED2CDC2CCC24AA
:100E10000E94242FA50194010E94652E6C0D7D1D5A
:100E20008E1D9F1D60937F057093800580938105C3
:100E300090938205C15001F7DD2309F450C005E805
:100E400015E0E801A12CB12C62E3C62ED12CE12CD7
:100E5000F12C8881882309F442C0B39419F40E94CC
:100E60007A063DC00E94242FA70196010E94652E9C
:100E7000E1E0E60FA5E8B5E08A2F801B8A1520F493
:100E80008D918E13F9CFE9CF2091840530E0A0E158
:100E9000B7E20E94FD2D9B01AC01AE2FB0E00E9495
:100EA0000C2E40907B0550907C0560907D057090E5
:100EB0007E05640D751D861D971D4090BB055090E5
:100EC000BC056090BD057090BE05461657066806C5
:100ED000790618F2E993A39488E1A812BACFCDB7A6
:100EE000DEB7E0E10C94A22E8436910520F4BC011B
:100EF00080E090E017C09C018E3B910528F42A55B4
:100F00003109AAE0B0E00CC0823D910528F4245BD1
:100F10003109A4E6B0E004C02D5C3109A8E5B2E0D7
:100F20000E94FD2DA4E6B0E09B01AC010E940C2EB6
:100F3000089590E08C599F4F0E947407089561E0D6
:100F400083E10E94982960E083E10E94D12982E038
:100F50008093B00085E08093B10061E083E00E945F
:100F6000982960E083E00E94D1290895A4E0B0E0D0
:100F7000ECEBF7E00C94942E009749F19C0140E0D3
:100F800050E068E478EE81E090E00E94652E61E038
:100F900083E129833A834B835C830E94D129298191
:100FA000822F3A81932F4B81A42F5C81B52F8F3FE5
:100FB0009105A105B10529F020F08FEF90E0A0E0A8
:100FC000B0E08093B3008091B000806107C060E022
:100FD00083E10E94D1298091B0008F7E8093B00080
:100FE0002496E2E00C94B02E60E08CE00E949829F8
:100FF00061E08BE00E94982961E08DE00E949829D1
:1010000060E082E00E94982961E084E00E949829D3
:10101000089542E050E068E476E080E00E941B28FA
:101020000895E3E0F0E089E080935700E491E670F2
:1010300081E0E63009F080E00895CF93DF93C82F78
:101040000E941108882381F0DFB781E08093720548
:10105000F8940E94570688E180936000C093600076
:10106000C1110E945706DFBFDF91CF9108958F9283
:101070009F92AF92BF92CF92DF92EF92FF92CF9367
:10108000FC01C0A5EC2FE770F0E0E658FC4FA08112
:10109000B0E0C7FF03C024E130E002C02FE030E041
:1010A000FC0197A183E1989FF0011124E25CFE4FBF
:1010B00080809180A280B380A20FB31F20E43FE123
:1010C0004DE750E00E94172EA50194010E94432E87
:1010D0008C2F887149F469017A01E0EDCE0EE7E0CA
:1010E000DE1EE11CF11C1BC0C7FF05C060E47AE8EE
:1010F0008CE29EE004C060E07EEE8AEB9BE069013A
:101100007A01F8EBCF0EFBE0DF1EE11CF11CA5011C
:1011100094010E94432EC20ED31EE41EF51EC70189
:10112000B60169517C4F8F4F9F4F28EE33E040E06E
:1011300050E00E94432EA8EEB3E00E940C2ECF9107
:10114000FF90EF90DF90CF90BF90AF909F908F90E7
:1011500008958F3F910551F048F0811522E09207E4
:1011600038F08115934030F482E0089580E00895CE
:1011700081E0089583E00895A0E0B0E0E2ECF8E0BB
:101180000C948F2EEB018A01B82FB695A0E0288130
:101190003981F80120832A813B8121832C813D8183
:1011A00022832E813F812383688179814A815B81FB
:1011B0002C813D81EE81FF819F2F9295990F990F90
:1011C000907C272F2370922B252F2370220F220F24
:1011D000922B232F23702295207F922BF80194834A
:1011E0000B5F1F4F2896AF5FBA1788F680FF24C0A9
:1011F000888199810E94A908D82E8A819B810E94AA
:10120000A908E82E8C819D810E94A908F82E8E8164
:101210009F810E94A908F0E4DF9EA001112490E1C3
:10122000E99E90011124242B282BE4E0FE9EB001BE
:101230001124262BF8012083CDB7DEB7E7E00C940C
:10124000AB2E803223E0920708F1883E23E092071C
:1012500040F48F519340E4E096958795EA95E1F745
:101260000895803D27E0920718F48C5D934008951F
:10127000883928E0920768F4885C974074E0969576
:1012800087957A95E1F78D509C4F089580E090E026
:1012900008958FEF93E008958C30910540F4A4E019
:1012A000880F991FAA95E1F7885D9C4F0895843FA8
:1012B00023E0920718F484529C4F0895811524E08E
:1012C000920740F48657934FF4E0880F991FFA95E0
:1012D000E1F7089580E998E008959C0136952795F7
:1012E00025753575821B930B9C012373337396957B
:1012F00087959695879583739373820F931F9C01AF
:1013000054E0369527955A95E1F7280F391F2F702D
:101310003F7041E051E0249FC001259F900D349F14
:10132000900D1124892F08952D98882319F000001D
:101330002B9A02C000002B9800002D9A00000895FF
:101340002D9A000083B12D98000082958170089538
:10135000CF93DF93D82F5C9A2D985C98C8E08D2F9F
:1013600080780E949409DD0FC150C9F72D98DF9154
:10137000CF9108958F770E94A8090895CF93DF93A6
:10138000D82FC8E08D2F80780E949409DD0FC150BE
:10139000C9F72D98DF91CF910895CF93DF932D98C2
:1013A000C8E080E0D82FDD0F0E94A0098D0FC1504A
:1013B000C9F7DF91CF9108950E94BA090E94CD0923
:1013C0005C9A0895A1E0B0E0E8EEF9E00C94942E68
:1013D000806869830E94A8096981862F0E94BE09DE
:1013E0005C9A2196E2E00C94B02ECF93C0917F05D9
:1013F000C827E82FF0E0EA58FA4F678589E70E948E
:10140000E2096C2F8DE30E94E2096C2F82E40E94B6
:10141000E209CF91089586E20E94DC090895CF93F6
:10142000DF93EC016C818CE10E94E2096D818DE11A
:101430000E94E2096E818EE10E94E2096F8180E2E2
:101440000E94E209688581E20E94E209698582E2E0
:101450000E94E2096A8583E20E94E2096B8584E2C8
:101460000E94E2096C8585E20E94E2096D858AE2AC
:101470000E94E2096E858EE60E94E2096F858FE682
:101480000E94E209688980E70E94E209698981E790
:101490000E94E2096A8982E70E94E209DF91CF9106
:1014A0000895CF92DF92EF92FF92CF93DF936B017B
:1014B0007C01C11488E3D8068CE9E8068CE1F806C3
:1014C00028F5C701B60120E836E948E950E00E9456
:1014D000432EE901689760E879E687E69FEF0E946E
:1014E0001F2E6C0D7D1D8E1D9F1DF2E0660F771F58
:1014F000881F991FFA95D1F721E732E040E050E0CC
:101500000E94432EF22EE32E80E421C0C701B601D3
:1015100020E03DE241E351E00E94432EE90168975B
:1015200060E073ED8EEC9EEF0E941F2E6C0D7D1D12
:101530008E1D9F1D660F771F881F991F21E732E0C0
:1015400040E050E00E94432EF22EE32E80E66C2F06
:101550006F71680F85E70E94E2096E2D86E70E9491
:10156000E2096F2D87E70E94E209DF91CF91FF909A
:10157000EF90DF90CF900895682F8DE60E94E209EA
:1015800008958F929F92AF92BF92CF92DF92EF9287
:10159000FF92CF93DF93D82F83E00E94DC098093E2
:1015A000710584E00E94DC098093700560E086E0AC
:1015B0000E94E20961E087E00E94E2096FE789E0AA
:1015C0000E94E20965E08AE00E94E20962E18BE0A4
:1015D0000E94E20965E18CE00E94E2096DEF8DE076
:1015E0000E94E20960E08EE00E94E209DD2319F02A
:1015F0008BE291E008C020919D0533E1239FC0015B
:101600001124825C9E4F0E940F0A6CE880E30E94C6
:10161000E2096FE082E30E94E20962E483E30E9450
:10162000E20980919E0587FF02C064E101C06AE083
:1016300084E30E94E2096AE285E30E94E2096DE226
:1016400086E30E94E20964ED87E30E94E20960E01C
:1016500088E30E94E20960E089E30E94E209D11177
:1016600009C0C0907F05D0908005E0908105F09082
:10167000820507C0C5E9CC2EC1ECDC2EED2CCEEDE9
:10168000FC2ECAE38F2C9924AA24BB24682D8C2F0E
:101690000E94E209682D85E08C0F0E94E209FE2C71
:1016A000ED2CDC2CCC24CF5FCE3361F76FEF83E4DD
:1016B0000E94E2096FEF84E40E94E2096FEF85E483
:1016C0000E94E2096FEF86E40E94E209DD2311F037
:1016D00066E002C0609183058DE60E94E20960E049
:1016E00089E70E94E209609184058AE70E94E20985
:1016F00060E083E70E94E20960E084E70E94E2097B
:10170000D11109C060917B0570917C0580917D05A8
:1017100090917E0504C060EC7AEC89E896E30E9423
:10172000510ADF91CF91FF90EF90DF90CF90BF9063
:10173000AF909F908F90089561E087E00E94E2094A
:1017400064E28EE70E94E20963E088E00E94E20919
:1017500060E088E00E94E20965E087E00E94E2091B
:1017600062E085E00E94E20983E00E94DC09809348
:10177000710584E00E94DC0980937005089583E080
:101780000E94DC098093710584E00E94DC0980934B
:10179000700561E087E00E94E2096AE070E080E0A5
:1017A00090E00E940E290E949C0B00000895CF92A9
:1017B000DF92FF920F931F93CF93DF931F92CDB7CA
:1017C000DEB7082F162F8EE399830E94E209F02ED0
:1017D000C02E9981D92E8C2D8F19811738F4F601DE
:1017E00061916F018FE70E94E209F5CF64E085E027
:1017F0000E94E20983E00E94DC098093710584E085
:101800000E94DC09809370050E94EB2860936C05B0
:1018100070936D0580936E0590936F0569E087E086
:101820000E94E20981E0809373050F90DF91CF91D0
:101830001F910F91FF90DF90CF9008950F931F930A
:101840000E94D70B80917305813099F40E94EB2898
:1018500000916C0510916D0520916E0530916F051A
:10186000601B710B820B930B603A764881409105A7
:1018700048F380917305813031F46EE971E082EEB6
:1018800095E00E94D72A1F910F9108950F931F93FF
:1018900080917305823021F41092730581E020C09D
:1018A000809173058130D9F40E94EB2800916C057A
:1018B00010916D0520916E0530916F05601B710BC5
:1018C000820B930B613A76488140910540F061E0CC
:1018D00087E00E94E2091092730582E001C080E077
:1018E0001F910F910895CF93DF93EC014AE050E0F0
:1018F0006D2F70E082EE95E00E94A52B6EE282EEE5
:1019000095E00E94A92ABE0184E0769567958A95A4
:10191000E1F76F7077274AE050E082EE95E00E9491
:10192000A52B6EE282EE95E00E94A92ABE016F709F
:1019300077274AE050E082EE95E00E94A52BDF91E8
:10194000CF910895D82FC0E0CD1790F45E9A409AB9
:1019500064E670E080E090E00E940E295E98409876
:1019600064E670E080E090E00E940E29CF5FECCF4B
:101970006CE271E080E090E00E940E29E4CF0F93CA
:101980001F93CF93DF93EC01062F15E0115051F018
:10199000CE010E94A030081741F0602FCE010E94B6
:1019A000A830F4CF82E00E94A20CDF91CF911F916A
:1019B0000F910895A0E0B0E0E0EEFCE00C94862EDC
:1019C000482E562EC0E0D0E0612C712CE12CF12C79
:1019D00000E010E041100CC06090D40586E4689EE1
:1019E0003001112459E1E52EF12C0AEB15E01EC05F
:1019F00091E049120FC06090D405E6E46E9E30017C
:101A00001124FBE16F0E711C49E2E42EF12C06E774
:101A100015E00CC082E0481209C028E1622E77244C
:101A20007394EE24E394F12C03ED15E043018C0E46
:101A30009D1E10927505109274053401A62CA818ED
:101A4000B12CC30101966C01AE14BF04A8F4A00E22
:101A5000B11E511006C0C3010E94A030F501808361
:101A600005C0F5016081C3010E94BF0CF5018081B2
:101A70000E9461063601E2CFC301511018C0C301B4
:101A80000E94A030B82EC6010E94A0302B2D30E05D
:101A9000322F2227282B809174059091750582178B
:101AA000930779F4C0E0D0E05524539493CF3601E6
:101AB000609175050E94BF0C60917405C6010E947B
:101AC000BF0CC05EDE4FC13E92E0D90708F482CF62
:101AD000852DCDB7DEB7E0E10C94A22E61E082E067
:101AE0000E94DA0C089560E082E00E94DA0C809196
:101AF000D305853020F01092D3050E946E0D8091A1
:101B0000D3058093D405089561E080E00E94DA0C4B
:101B100061E081E00E94DA0C089560E080E00E94BC
:101B2000DA0C882351F060E081E00E94DA0C88230F
:101B300021F080917605883349F00E94BF060E940B
:101B40007A0681E00E94DF060E94840D08958823B2
:101B500019F06AEA71E002C06EEA71E082EE95E087
:101B60000E94D72A0895FF920F931F93CF93DF937C
:101B700069EC7BE082EE95E00E94832A40917B0530
:101B800050917C0560917D0570917E052AE030E0E2
:101B900082EE95E00E94AC2B63EB7BE082EE95E059
:101BA0000E94832A40917F055091800560918105B4
:101BB0007091820520E130E082EE95E00E94AC2B2E
:101BC0006DE97BE082EE95E00E94832A4AE050E0D6
:101BD0006091830582EE95E00E94D42B67E87BE05C
:101BE00082EE95E00E94832A4AE050E060918405ED
:101BF00082EE95E00E94D42B61E77BE082EE95E0D7
:101C00000E94832AC5E8D5E0F12C8E0188818823C3
:101C1000A9F0FF2031F061EB71E082EE95E00E94C7
:101C2000A62A21964AE050E0F801608182EE95E014
:101C30000E949D2BF394F8E1FF12E7CF82EE95E02E
:101C40000E94B12A6BE57BE082EE95E00E94832A38
:101C50004AE050E060919D0582EE95E00E94D42B11
:101C600066E47BE082EE95E00E94832AE0919E0587
:101C7000E770F0E0EE0FFF1FEE57FC4F60817181BF
:101C800082EE95E00E94D72A61E37BE082EE95E048
:101C90000E94832A80919E058871883069F028F41B
:101CA000811113C068E27BE00CC0803141F08831C3
:101CB00061F46CE07BE005C06CE17BE002C066E1B2
:101CC0007BE082EE95E00E94C52A68EF7AE082EE22
:101CD00095E00E94832A40917705509178056091A4
:101CE000790570917A052AE030E082EE95E00E9455
:101CF000AC2B6FED7AE082EE95E00E94832A809112
:101D0000BF0580710E94A70D66EC7AE082EE95E037
:101D10000E94832A8091BF0580740E94A70D6DEAFE
:101D20007AE082EE95E00E94832A8091BF0580725E
:101D30000E94A70D60E97AE082EE95E00E94832A76
:101D400086E795E00E943708AB01BC012AE030E04D
:101D500082EE95E00E948E2B6BE87AE082EE95E0B1
:101D60000E94832A86E795E00E9437089B01AC0118
:101D700060E472E48FE090E00E94432EBA01A90172
:101D80002AE030E082EE95E00E948E2B68E87AE04F
:101D900082EE95E00E94C52ACDB7DEB7E5E00C944F
:101DA000AD2E8F929F92AF92BF92CF92DF92EF9221
:101DB000FF92811107C06FE77AE082EE95E00E9402
:101DC000C52A2FC090E00E94740724E630E040E06E
:101DD00050E00E94432ECA01B9012AE030E040E001
:101DE00050E00E94432E49015A016B017C012AE018
:101DF00030E0B501A40182EE95E00E948E2B6EE2E8
:101E000082EE95E00E94A92A2AE030E0B701A601FF
:101E100082EE95E00E948E2B63E782EE95E00E94B1
:101E2000E92AFF90EF90DF90CF90BF90AF909F9006
:101E30008F9008951F93CF93DF9365E77AE082EE4A
:101E400095E00E94832A80919F05813041F46CE5E2
:101E50007AE082EE95E00E94C52A10E050C0823000
:101E600019F465E47AE0F5CF843019F461E37AE09F
:101E7000F0CF853091F766E27AE0EBCFC12FD0E06A
:101E8000C930D1050CF441C068E3610F82EE95E0E2
:101E90000E94A92A6EE17AE082EE95E00E94832AF0
:101EA000BE016F5F7F4F4AE050E082EE95E00E94F6
:101EB0006D2B63E17AE082EE95E00E94832AC156A1
:101EC000DA4FE981E03218F566E07AE082EE95E0DB
:101ED0000E94832A8981803130F06DE673E082EEC2
:101EE00095E00E94A62A69816F7070E06F5F7F4F56
:101EF0004AE050E082EE95E00E94762B1F5F8091D1
:101F00004805181708F4BACF0FC061E3BECFEF70D1
:101F1000F0E0EE0FFF1FEE56FC4F6081718182EE04
:101F200095E00E94D72AEACF6BEE79E082EE95E049
:101F30000E94832A8091B7050E94D10E60ED79E05E
:101F400082EE95E00E94832A8091B8050E94D10E0E
:101F500065EB79E082EE95E00E94832A8091B905D5
:101F60000E94D10E6AE979E082EE95E00E94832A10
:101F70004091AF055091B0056091B1057091B205E7
:101F8000411551056105710539F12AE030E082EE15
:101F900095E00E94AC2B67E679E082EE95E00E9426
:101FA000832A8091B3050E949907AB01BC012AE006
:101FB00030E082EE95E00E94AC2B63E479E082EEA3
:101FC00095E00E94832A4AE050E06091B40582EED9
:101FD00095E00E94D42B06C06AE379E082EE95E09A
:101FE0000E94C52A6DE179E082EE95E00E94832A85
:101FF0006091B5057091B6054AE050E082EE95E03B
:102000000E94BE2B60E079E082EE95E00E94832A78
:102010006091AE05603450F470E06F5F7F4F4AE02E
:1020200050E082EE95E00E94762B06C067EF78E0E4
:1020300082EE95E00E94C52A6AED78E082EE95E096
:102040000E94832A8091AD0580FF03C063EB71E09D
:1020500002C067EB71E082EE95E00E94D72A6DEB3B
:1020600078E082EE95E00E94832A8091AD0582702F
:102070000E94A70D6EE978E082EE95E00E94832A27
:102080008091AD0584700E94A70D6FE778E082EE25
:1020900095E00E94832A8091AD0588700E94A70D6B
:1020A000DF91CF911F9108950F931F93CF93DF93EB
:1020B000209145052F3FA9F56FEF75E082EE95E081
:1020C0000E94832A85E893E00E94730C6EED75E010
:1020D00082EE95E00E94832A809146059091470503
:1020E0000E94730C6BEA75E082EE95E00E94C52AAF
:1020F00068E875E082EE95E00E94C52A60E775E029
:1021000082EE95E00E94C52A6BE475E082EE95E0D0
:102110000E94C52A82EE95E00E94B12A0E941A0F01
:1021200068C012160CF065C0332727FD30958091EA
:10213000480590E0821793070CF45BC066E375E0F6
:1021400082EE95E00E94832A60914505772767FD1E
:1021500070954AE050E082EE95E00E94762B6BE0AD
:1021600075E082EE95E00E94832A10E008E28091FB
:1021700049051817D0F5C12FD0E0CC0FDD1FC65B85
:10218000DA4F288130E080914505992787FD9095A9
:1021900001972817390739F56BEB71E082EE95E06E
:1021A0000E94A62A4AE050E0602F82EE95E00E944D
:1021B0009D2B6FEB71E082EE95E00E94A62AE981EB
:1021C000EF70F0E0EE0FFF1FEE56FC4F6081718163
:1021D00082EE95E00E94A62A63EC71E082EE95E023
:1021E0000E94A62A0F5F1F5FC2CF82EE95E00E9479
:1021F000B12ADF91CF911F910F910895FF920F9314
:102200001F93CF93DF93C5E8D5E0F12C8E01888131
:102210008823D1F165EC71E082EE95E00E94A62A58
:102220004AE050E06F2D82EE95E00E949D2B62ED1A
:1022300071E082EE95E00E94A62A2196F8012081A5
:1022400030E0A0E1B7E20E94FD2D9B01AC01A0911E
:102250008405B0E00E940C2EAB01BC0180917B058F
:1022600090917C05A0917D05B0917E05480F591F86
:102270006A1F7B1F2AE030E082EE95E00E94AC2BC3
:10228000F394F8E1FF12C2CFCDB7DEB7E5E00C94CE
:10229000AD2E1092DF0485E6E0EEF4E0DF011D9242
:1022A0008A95E9F70895CF93C82F8F3719F08830B2
:1022B00009F045C0E091DF04EE23D9F1E150E0934D
:1022C000DF04F0E0E052FB4F10826DE070E082EE40
:1022D00095E00E945906C0E08091DF04C81760F4C1
:1022E000EC2FF0E0E052FB4F608170E082EE95E071
:1022F0000E945906CF5FF0CF60E270E082EE95E079
:102300000E9459066DE070E082EE95E00E94590649
:10231000C0E08091DF04C81778F5EC2FF0E0E052C0
:10232000FB4F608170E082EE95E00E945906CF5F1E
:10233000F0CF67E082EE95E00E94A92A1DC08B31A4
:1023400019F40E9449111AC08D30C1F08A30B1F0E1
:102350008091DF04843668F76C2F70E082EE95E0A0
:102360000E945906E091DF0481E08E0F8093DF0424
:10237000F0E0E052FB4FC08380E001C081E0CF91EC
:102380000895CF93C82F0E94EB286093C8047093E0
:10239000C9048093CA049093CB04C093DD04CC237A
:1023A00029F040E051EE60E070E004C040E855E202
:1023B00060E070E082EE95E00E94332DCF910895A9
:1023C0009091CC04492F4F7050E0BA016F5F7F4F5E
:1023D000292F30E0E4E035952795EA95E1F762177B
:1023E000730759F0FA01E353FB4F808381E0890FB3
:1023F0008F70907F892B8093CC0408956EE770E0F6
:1024000082EE95E00E9459060895A3E1B1E0EBE069
:10241000F2E10C94872EE5E8F5E0712C8191882398
:1024200021F0739428E17212F9CF66ED71E082EE2B
:1024300095E00E94D72A4AE050E0672D82EE95E0B1
:102440000E94D42B80E00E94C10A0E949C0B8E0146
:102450000E5F1F4FC12CD12C7601C39466246A9461
:102460005C2C0E94DF284B015C012091840530E048
:10247000A0E1B7E20E94FD2D9B01AC01C701B601AE
:102480000E941F2E20917B0530917C0540917D0597
:1024900050917E05620F731F841F951F2091BB050D
:1024A0003091BC054091BD055091BE0526173707F8
:1024B0004807590718F4F801608229C08C2D0E9442
:1024C000F50961E070E080E090E00E940E29F801DB
:1024D00010820E94DF28681979098A099B09643FE4
:1024E00071408105910540F40E940B0AF80190812A
:1024F000981778F78083EDCF50FE05C05D9841981E
:102500005E9A409A04C05D9A419A5E9840982FEF77
:10251000C21AD20AE20AF20A0F5F1F4F8FEFC816E3
:10252000D104E104F10409F09BCFCE019395FC01A5
:10253000D82E7FEF68EC2E2F281B271510F051E0C6
:1025400056C0DE01129651E02FEF41E03D91321767
:1025500010F0322F01C0452F5F5F5F3F11F0232F36
:10256000F5CF4193242F30E0A1E0B0E0AC0FBD1FC8
:10257000A20FB31F5C93413079F0DE01A20FB31FAD
:102580005C93423049F0AFEFBFEFAC0FBD1FA20F1D
:10259000B31F6C934E3F78F6A2E0B0E0AC0FBD1FC6
:1025A000A20FB31F7C934D3F30F6A3E0B0E0AC0F19
:1025B000BD1FA20FB31F6C93BECF452F242F30E059
:1025C000FC01E20FF31F6081AFEFB0E0AC0FBD1F65
:1025D000A20FB31F2C91621748F44150DC01A40FE5
:1025E000B11D2C9120836C934111E8CF5F5F57158B
:1025F00020F3372D369520E0231770F4DC01A20F6D
:10260000B11D4C91522F530FFC01E50FF11D50816C
:102610005C9340832E5FF0CFF5E8EF2EF5E0FF2EC0
:102620008C01802F8D19871598F4F801C1908F01C6
:102630004AE050E06C2D82EE95E00E949D2B6CE20A
:1026400082EE95E00E94A92AF701C1927F01E9CFAD
:1026500082EE95E00E94B12A81E0CD5EDE4FEFE090
:102660000C94A32E1F920F920FB60F9211241F935A
:102670002F933F934F935F936F937F938F939F938A
:10268000AF93BF93CF93DF93EF93FF93C0918600F7
:10269000D091870080918704909188042091A904AB
:1026A000211155C09E01281B390B8091BF059091C7
:1026B000C005A091C105B091C20585FD02C0369547
:1026C0002795253C49E03407B8F140910A0150E0D4
:1026D00060E070E02CE1B695A795979587952A95CF
:1026E000D1F70097A105B10521F481E090E0A0E0C9
:1026F000B0E084179507A607B707D8F480910A01C0
:102700008F3FB9F040E080910A01481780F4842F90
:1027100090E0880F991FFC01E757FB4F2081318122
:10272000FC01E55FFE4F318320834F5FECCF1092B9
:10273000AA0410920A010BC02D3B82E0380720F05A
:1027400080910A018031D8F08FEF80930A01D093F5
:102750008804C0938704FF91EF91DF91CF91BF91DF
:10276000AF919F918F917F916F915F914F913F9129
:102770002F911F910F900FBE0F901F9018951091E1
:102780000A0181E0810F80930A01C9010E94210999
:10279000E12FF0E0EE0FFF1FE757FB4F918380839F
:1027A000D6CF83E0809380008AE980938100809176
:1027B000BF0586FD05C08091810080648093810003
:1027C0008FEF9FEF909389008093880080916F0036
:1027D000806280936F0008950E94730D8091D405EC
:1027E000843011F41092D40508956F3018F0869556
:1027F0008058089589E0689F802D11240895A0E0F5
:10280000B0E0E5E0F4E10C948E2EC82F0E94EB2896
:10281000009138041091390420913A0430913B041E
:102820006B017C01C01AD10AE20AF30A9701860102
:1028300049E8C41643E1D406E104F10410F0109213
:102840003C04609338047093390480933A04909365
:102850003B042091A9048FEF820F8230D8F5E091DC
:102860003C04EE2309F44EC1E13011F482E0B8C11A
:10287000E03108F034C181E08E0F80933C04F0E039
:10288000E757FB4FC083803109F0ACC1EBE8F4E0BF
:10289000213029F4A181A695A695808108C0808168
:1028A0009181A92FA695A695A69596958795A03175
:1028B00048F4B0E090E0AA0FBB1FA55FBE4F119691
:1028C0009C938E931092AA04329684E0E939F8071B
:1028D000F9F688C1233009F005C1E0913C04E1110B
:1028E00004C0CF3009F07EC10DC1E83148F481E069
:1028F0008E0F80933C04F0E0E857FB4FC08372C119
:10290000E83109F0ECC0C111EAC040E050E0ABE0B2
:10291000CA01B3E0880F991FBA95E1F7A49F90010F
:10292000A59F300D1124F901E757FB4F6081E1812C
:102930007E2F777075956795FC01EE0FFF1FE55FA1
:10294000FE4F71836083F901E657FB4FB081B69566
:10295000B695B695E181FE2FF295FF0FF07E6F2FB1
:102960006B2BE695E695E6957E2F777075956795C6
:10297000FC01EE0FFF1FE35FFE4F71836083F901DF
:10298000E557FB4FB081B295B695B695B370C1814E
:10299000DC2FDD0FDD0F6D2F6B2BC295C695C69515
:1029A000C370E281E170EE0FEE0F7E2F7C2B7595E8
:1029B0006795FC01EE0FFF1FE15FFE4F718360839F
:1029C000F901E357FB4FB081B695E181FE2FF795F2
:1029D000FF27F7956F2F6B2BE6957E2F77707595F8
:1029E0006795FC01EE0FFF1FEF5EFE4F7183608362
:1029F000F901E257FB4FB081B295BF70E181FE2F24
:102A0000F295F07F6F2F6B2BE295EF707E2F777032
:102A100075956795FC01EE0FFF1FED5EFE4F71830C
:102A20006083F901E157FB4FB081BB1FBB27BB1F80
:102A3000C181DC2FDD0F6D2F6B2BCC1FCC27CC1F62
:102A4000E281E370EE0F7E2F7C2B75956795FC017C
:102A5000EE0FFF1FEB5EFE4F71836083F901EF56AF
:102A6000FB4FB081B695B695E181FE2FF295FF0F31
:102A7000FF0FF07C6F2F6B2BE695E6957E2F77701E
:102A800075956795FC01EE0FFF1FE95EFE4F7183A0
:102A90006083F901EE56FB4F208122952695277021
:102AA0003181E32FEE0FEE0FEE0F6E2F622B732F9F
:102AB00072957695777075956795FC01EE0FFF1FFF
:102AC000E75EFE4F718360834F5F5F4F4230510579
:102AD00009F01ECF80919F0483FF1092AA041092E8
:102AE0003C0480C0243009F07DC060913C04611139
:102AF0000BC0C83AB1F4109275051092740588EABB
:102B00000E94610681E06CC0613019F4C093370403
:102B100004C0623031F4C09336048C2F0E946106E9
:102B20005AC0E09136042E2F30E0220F331F462F7B
:102B300050E0C9010296841795073CF0633268F7AC
:102B4000FA01EA57FB4FC083E8CF2D5F3F4F8C2F30
:102B500090E060917405709175054217530749F430
:102B6000982F88278627972790937505809374055B
:102B700032C06817790769F580913704813049F5CB
:102B8000E13118F080E180933604F0903604CAE811
:102B9000D4E000E010E00F15D0F4FE013197808101
:102BA00090E0982F88272881822B63E0969587955F
:102BB0006A95E1F70E942109F801EE0FFF1FE55F1A
:102BC000FE4F918380830F5F1F4F2296E4CF1092B8
:102BD000AA0410923C0480913C04882319F08F5F72
:102BE00080933C04CDB7DEB7E8E00C94AA2EE82F22
:102BF000F0E0E654FA4FE185E03150F4F894F0E06B
:102C0000EE0FFF1FE55FFE4F80819181789408955C
:102C10008EE08E0F8B3058F4F0E0E25FF10924E68D
:102C20002E9FC0012F9F900D11240C960895E03F18
:102C3000F1F028F4E03161F0E13161F006C0ED3FE0
:102C400081F0EE3F89F0E13F49F080E092E00895A5
:102C500082E101C083E10E942D2A089586E090E080
:102C600008958AEF93E008958FEF93E0089580E050
:102C700090E00895A2E2B0E0E0E4F6E10C94842E46
:102C80009E012F5F3F4F80E1D9011D928A95E9F7A0
:102C900064E072E082EE95E029A33AA30E94D72A6D
:102CA0000E94BF0B1D8A1E8A1F8A188E312C212C70
:102CB00000E0812C912C540170EC472E7DE9572EB9
:102CC00078E5672E75E3772EE0E5CE2EE3ECDE2E79
:102CD000E12CF12C84EF91E0A0E0B0E08D8F9E8F8D
:102CE000AF8FB8A380EC97EFAAEBB7E3898F9A8FE9
:102CF000AB8FBC8F80EC9DE9A8E5B5E3898B9A8BFF
:102D0000AB8BBC8B82EE95E00E94EB2B892B09F4F8
:102D1000E1C082EE95E00E94182C9C0133272C32F2
:102D2000310509F442C0ACF42332310509F0ABC0DF
:102D300019821A821B821C821D821E821F821886A3
:102D400019861A861B861C861D861E861F86188A73
:102D500060C02434310529F02335310509F4B2C0AF
:102D600092C064E482EE95E00E94A92A2AE030E055
:102D700040EC5DE968E575E382EE95E00E94372B53
:102D80006CE282EE95E00E94A92A2AE030E040EC55
:102D900057EF6AEB77E382EE95E00E94372B6CE207
:102DA00082EE95E00E94E92AADCF0F5F043009F072
:102DB000A9CF29813A814B815C81A8EEB3E00E94C2
:102DC0000C2E698B7A8B8B8B9C8B2D813E814F8156
:102DD00058850E940C2E698F7A8F8B8F9C8F298546
:102DE0003A854B855C852D8F3E8F4F8F58A32D855F
:102DF0003E854F8558890E940C2E6B017C01603204
:102E00003EE473078105910530F462E38CE10E9492
:102E1000E20900E077CF603345E77407810591054B
:102E200010F462E2F3CF60345CE975078105910527
:102E300010F466E2EBCF80E5C81683ECD806E10417
:102E4000F10410F462E1E2CF90E6C9169AEED906D9
:102E5000E104F10410F465E1D9CFA0E7CA16A1E1BD
:102E6000DA06A1E0EA06F10410F461E0CFCFB0EA9F
:102E7000CB16B6E8DB06B1E0EB06F10410F463E034
:102E8000C5CF65E0C3CF10ED180F1A3008F03ACF68
:102E9000E1E0F0E0EC0FFD1F24E0029FE00DF11DEA
:102EA00011242081318142815381AAE0B0E00E9447
:102EB0000C2E610F711D811D911D608371838283B2
:102EC000938320CF49885A886B887C88812C912CE9
:102ED000540118CF81149104A104B10489F4C301F1
:102EE000B2010E94510A61E070E080E090E00E942F
:102EF0000E291D8A1E8A1F8A188E312C22242A949C
:102F00008D8D9E8DAF8DB8A188169906AA06BB0639
:102F1000D0F40E940B0A2D893E894F89588D280FC5
:102F2000311D411D511D2D8B3E8B4F8B588F3816F7
:102F300008F4382E821508F4282E3FEF831A930ADE
:102F4000A30AB30A56C0C301B20128EE33E040E041
:102F500050E00E94432EBA01A9012AE030E082EE3F
:102F600095E00E948E2B6CE282EE95E00E94A92AE9
:102F70004AE050E0632D82EE95E00E949D2B6CE2CA
:102F800082EE95E00E94A92A6D897E898F89988DAD
:102F9000A50194010E94432EBA01A9012AE030E064
:102FA00082EE95E00E948E2B6CE282EE95E00E940C
:102FB000A92A4AE050E0622D82EE95E00E949D2B06
:102FC0006CE282EE95E00E94E92A4C0C5D1C6E1CBE
:102FD0007F1C898D9A8DAB8DBC8D84159505A605BA
:102FE000B70520F449885A886B887C88812C912CFD
:102FF000540129893A894B895C89283E334041052F
:10300000510509F07FCEA296E2E10C94A02EACE12E
:10301000B0E0EDE0F8E10C948E2E0E94EB286B01FD
:103020007C0181E00E94C10A14E703E0198361E09A
:10303000CE0101960E941E0C009373050E949C0B0A
:103040006AEF70E080E090E00E940E2980917305A5
:10305000833089F482EE95E00E94EB2B892B59F4A2
:103060000E94EB286C197D098E099F096038734C0A
:10307000894C9140D8F280917305833009F44FC098
:103080008FE70E94BA090E94CD098983843511F027
:1030900083E05CC00E94CD091092460580934705ED
:1030A0000E94CD092091460530914705280F311D1A
:1030B00030934705209346050E94CD09809348052B
:1030C0000E94CD0980934905813110F7F12C0F2D15
:1030D00010E08091490590E0880F991F08171907A3
:1030E00040F40E94CD09F801E65BFA4F8083F39427
:1030F000EECF80E7898361E0CE0101960E941E0C2D
:1031000083E0809373050E949C0B62E370E080E093
:1031100090E00E940E2980917305833011F482E0C3
:1031200015C08FE70E94BA090E94CD0989838035B6
:1031300009F0AECF0FE915E00E94CD09F8018193A7
:103140008F01F5E00A3B1F07B9F781E06C96E8E0D4
:103150000C94AA2E80914505992787FD9095A92F5B
:10316000B92FFC013196EB30F10508F066C0EC5C3C
:10317000FF4F0C94BB2E62E778E082EE95E00E9450
:10318000C52A85E893E00E94730C6AE578E082EE38
:1031900095E00E94C52A65E378E082EE95E00E9402
:1031A000C52A6BE078E082EE95E00E94C52A6AEEBF
:1031B00077E082EE95E00E94C52A6DEB77E082EE23
:1031C00095E00E94C52A67E977E082EE95E00E94CB
:1031D000C52A63E777E082EE95E00E94C52A6CE499
:1031E00077E082EE95E00E94C52A82EE95E00E948B
:1031F000B12A0E94B30D21C06FE277E01AC06AE0E5
:1032000077E017C065EF76E014C066ED76E011C098
:1032100062E976E00EC06DE776E00BC068E676E026
:1032200082EE95E00E94C52A62E276E002C06CE080
:1032300076E082EE95E00E94C52A6AE070E080E0C8
:1032400090E00E940E2982EE95E00E94EB2B892BE4
:1032500029F082EE95E00E94182CF5CF0895ACE19C
:10326000B0E0E5E3F9E10C948E2E909145059F3F87
:1032700009F023C1482F50E0FA013A97EF36F105E3
:1032800008F00FC1E15CFF4F0C94BB2E61E172E0CE
:10329000A0C06DE172E082EE95E00E94D72A85E73A
:1032A00089838BE1EFE9F5E0DE01129601900D9242
:1032B0008A95E1F76CE1CE0101960E941E0C0E94F6
:1032C0009C0B83E08093730568EC70E080E090E0F5
:1032D0000E940E2980917305843009F0E2C08FE7C7
:1032E0000E94BA090E94CD098983853509F0D9C0A9
:1032F0006DEE74E082EE95E00E94C52A6FEC74E0FA
:1033000082EE95E00E94C52A61EB74E096C065E309
:1033100072E082EE95E00E94D72A89E6898361E017
:10332000CE0101960E941E0C0E949C0B83E08093AC
:10333000730568EC70E080E090E00E940E298091B7
:103340007305843009F0ADC08FE70E94BA090E946E
:10335000CD0989838E010E5F1F4F7E014DE1E40E82
:10336000F11C0E94CD09F80181938F01EE15FF0534
:10337000C1F78BE1FE013296AFE9B5E001900D9205
:103380008A95E1F78981893409F08BC063E974E09B
:1033900082EE95E00E94C52A65E774E082EE95E032
:1033A0000E94C52A67E574E048C06FE472E082EECF
:1033B00095E00E94D72A8EEF8093450572C0805217
:1033C0008750805390914805981708F066C06EE5C5
:1033D00072E082EE95E00E94D72A63C084E1809378
:1033E000450560E274E029C085E18093450569EEFA
:1033F00073E023C086E18093450562EB73E01DC056
:1034000087E18093450568E673E017C088E1809303
:10341000450567E573E011C089E18093450563E4E4
:1034200073E00BC08AE1809345056EE273E005C04E
:103430008BE18093450566E073E082EE95E00E94A3
:10344000C52A2FC06CEE72E082EE95E00E94C52A7C
:103450008091AD0591E01DC066ED72E082EE95E0D1
:103460000E94C52A8091AD0592E013C061EC72E024
:1034700082EE95E00E94C52A8091AD0594E009C0D6
:1034800066EA72E082EE95E00E94C52A8091AD0561
:1034900098E089278093AD058FEF809345050E94C2
:1034A000541082EE95E00E94EB2B892B09F45BC14E
:1034B00082EE95E00E94182CF4CF0E9453118823CD
:1034C00009F451C18091DF04811104C08FEF809312
:1034D000450541C140E050E060E070E080EE94E0DE
:1034E0000E94322F40914505042F112707FD1095AA
:1034F000212F312FF8013197EB31F10508F01BC175
:10350000E255FF4F0C94BB2E552747FD5095209157
:10351000480530E0241735070CF40DC18B019C01E0
:103520000150110921093109003211052105310528
:1035300058F0C0904905EBE4F5E0F12CD12CA8E25D
:10354000EA2E415051090FC0FA01E156FA4F61507D
:103550006083D9C0DF0111972C9130E02417350723
:1035600029F0F3943296FC10F5CFCBC00E2D10E06D
:1035700020E030E0061717072807390741F42081BB
:10358000DA01A156BA4F11962C93DD24D394E3941B
:10359000E8CF6F3F71058105910511F008F0CBC0B0
:1035A0006093B705B0C06F3F71058105910511F0BB
:1035B00008F0C1C06093B805A6C06F3F71058105D2
:1035C000910511F008F0B7C06093B9059CC0209137
:1035D000E00420622037E9F440E050E060E070E071
:1035E00081EE94E00E94322F9B01AC01DC01CB0103
:1035F0000197A109B1090897A105B10508F0AEC06E
:10360000A4EDB0E30E940C2E6A5E7C4A8A46954E79
:1036100024C02636E9F440E050E060E070E081EE3E
:1036200094E00E94322F9B01AC01DC01CB01019799
:10363000A109B1090797A105B10508F08FC0A8EA53
:10364000B1E60E940C2E645E7C438E46944E05C00B
:10365000611571058105910579F08B019C01005C74
:103660001D49284535430130FAE51F07F2E62F07CB
:10367000F2E03F0708F05FC06093AF057093B005BC
:103680008093B1059093B2053EC06F3F71058105EF
:10369000910511F008F04FC06093B30534C08B0161
:1036A0009C0101501109210931090F3F1105210524
:1036B000310508F040C06093B40525C08B019C0122
:1036C000045C1940210931090D344DE1140721052D
:1036D000310528F47093B6056093B50514C06115E3
:1036E00071058105910521F48FEF8093AE050BC024
:1036F0006134710581059105F0F461506093AE0568
:1037000002C0DD20C1F08091DE0481111AC08091D9
:103710007F0590918005A0918105B0918205019669
:10372000A11DB11D80937F0590938005A093810515
:10373000B093820506C060E772E082EE95E00E94D9
:10374000D72A0E9449118FEF809345056AE082EEE7
:1037500095E00E94E92A0E94541005C061E070E0E3
:1037600080E090E07ACF6C96E8E00C94AA2E6AE5AF
:1037700072E082EE95E00E94C52A62E472E082EE79
:1037800095E00E94C52A82EE95E00E94EB2B892BE2
:1037900031F082EE95E00E94182C0E942F190E94B1
:1037A0000718823029F0833051F46DE072E002C0D6
:1037B00064E272E082EE95E00E94C52A08958FEFE0
:1037C000809345051092DE040E94541080914505B7
:1037D0008E3F69F082EE95E00E94EB2B892BB1F3CE
:1037E00082EE95E00E94182C0E942F19EFCF0895C9
:1037F0000F931F93109145051F3F09F0D2C08934E4
:1038000009F457C000F5883309F469C058F48033CF
:1038100009F477C008F061C08B3109F440C08132EF
:10382000B1F1B9C0813409F487C030F4893309F4A7
:1038300066C0803461F1AFC0823409F48EC0863432
:1038400009F448C0A8C0823609F487C078F48835E6
:1038500031F128F48235C1F18335E1F09CC08A351D
:1038600009F494C0813609F467C095C0823761F1CC
:1038700028F4863679F18936E1F08DC0883779F001
:103880008A3709F483C0833709F085C003C061E13A
:1038900072E015C00E94840D6EE872E004C00E94C0
:1038A0008D0D68EA72E082EE95E00E94D72A8EEFD5
:1038B00070C00E947A060E94BF0667EC72E082EE3A
:1038C00095E00E94D72A67C081E00E94DF0660EE83
:1038D00072E0F5CF0E94FE105EC080535AC06AEFBE
:1038E00071E082EE95E00E94C52A90919E0588E0E5
:1038F000890F8871977E892B80939E051AC089E075
:1039000048C067EE71E082EE95E00E94C52A809182
:10391000BF059091C005A091C105B091C20520E1FD
:1039200082278093BF059093C005A093C105B093F3
:10393000C205109345052FC061ED71E082EE95E060
:103940000E94C52A8091BF059091C005A091C10534
:10395000B091C20540E4842710C060EC71E082EEB3
:1039600095E00E94C52A8091BF059091C005A09165
:10397000C105B091C20520E282278093BF059093D4
:10398000C005A093C105B093C20502C00E94B71B39
:103990008FEF80934505809145058E3F09F0D4C097
:1039A000DDC00E945311882309F4D8C08091DF0440
:1039B000811104C08FEF80934505C6C040E050E000
:1039C00060E070E080EE94E00E94322F00914505A7
:1039D000112707FD1095212F312FF8013197E9307C
:1039E000F10508F0B4C0E753FF4F0C94BB2E8B01D8
:1039F0009C01015C1D49284535430F3F194522466E
:103A0000324008F0A4C060937B0570937C058093DE
:103A10007D0590937E0577C060937F057093800548
:103A2000809381059093820581E08093DE046BC0D2
:103A3000683071058105910508F089C060938305A0
:103A400062C08B019C0101501109210931090A3022
:103A500011052105310508F07AC06093840553C033
:103A600061EB71E080EE94E00E946C3010E0009712
:103A700099F00E944630009779F0183130F4E12F28
:103A8000F0E0EA58FA4F87871F5F61EB71E080E052
:103A900090E00E946C30EBCF1831A8F5E12FF0E0F8
:103AA000EA58FA4F17861F5FF7CF65307105810519
:103AB000910508F04CC060939D0525C08B019C01C9
:103AC000015011092109310906301105210531057F
:103AD000F0F520919E05287F262B20939E0513C08C
:103AE0008B019C0101501109210931090115124C6A
:103AF0002140310560F560937705709378058093D8
:103B0000790590937A058091DE04811113C080912C
:103B10007F0590918005A0918105B0918205019665
:103B2000A11DB11D80937F0590938005A093810511
:103B3000B09382050E9449118FEF809345056AE09A
:103B400082EE95E00E94E92A0E94AA1807C060E769
:103B500072E082EE95E00E94D72AECCF1F910F9180
:103B600008958FEF809345051092DE040E94AA18F5
:103B7000809145058E3F69F082EE95E00E94EB2B27
:103B8000892BB1F382EE95E00E94182C0E94F81B5D
:103B9000EFCF6AE070E080E090E00E940E2982EEB4
:103BA00095E00E94EB2B892B29F082EE95E00E9494
:103BB000182CF5CF0895CF93C82F682F82EE95E08B
:103BC0000E94452C90916A059C2790936A05CF919D
:103BD0000895A1E0B0E0EFEEFDE10C94942E9983FE
:103BE0000E94DB1D9981892F0E94DB1D2196E2E056
:103BF0000C94B02E1F93CF93DF93182FEB011092EC
:103C00006A0565EB70E082EE95E00E94590662E677
:103C100070E082EE95E00E945906812F0E94DB1D24
:103C2000CE010E94E91DDF91CF911F91089560910F
:103C30006A0582EE95E00E94452C0895A1E2B0E06D
:103C4000E4E2FEE10C94902E7B018A018C3009F4B1
:103C500053C108F040C0863009F4BCC018F5833069
:103C600009F491C070F4813009F472C0823009F017
:103C700048C26BE170E082E00E94FA1D0FE915E096
:103C800078C0843009F487C0853009F03AC2609169
:103C9000490570E0660F771F85E00E94FA1D0AE46F
:103CA00015E086C0893009F4A7C070F4873009F4A4
:103CB0009BC0883009F025C261E070E088E00E9476
:103CC000FA1D8091D40523C28A3009F4CAC08B3012
:103CD00009F4F2C016C28A3609F475C1D8F48736E1
:103CE00009F43AC138F4853609F40EC1863609F470
:103CF0001FC107C2883609F437C1893609F001C2ED
:103D000061E070E089E60E94FA1D0E947A060E9436
:103D1000BF06F5C18D3609F4D4C138F48B3609F4E9
:103D200091C18C3609F49AC1ECC18E3609F4DCC11C
:103D3000873C09F0E6C161E070E087EC0E94FA1D63
:103D400081E00E94DB1D0E94171E10926B05E3C1EB
:103D500069E270E081E00E94FA1D06E715E0F801D3
:103D600081918F010E94DB1DF5E00F391F07B9F724
:103D7000D0C1F80181918F010E94DB1DF5E00A3B63
:103D80001F07B9F7C6C161E070E083E00E94FA1D29
:103D90000E940718BCC161E070E084E00E94FA1D37
:103DA00081E00E94DB1D0E94171E0E943A16B3C1DB
:103DB0008091490590E0880F991F98012A54354059
:103DC0002817390708F0A5C1F80181918F010E94D9
:103DD000DB1DEECF62E070E086E00E94FA1D85E810
:103DE00093E00E94E91D95C161E070E087E00E94C8
:103DF000FA1D809148058BC186E6898361E0CE017A
:103E000001960E941E0C0E949C0B83E08093730518
:103E100068EC70E080E090E00E940E2980917305CC
:103E20008430D9F48FE70E94BA090E94CD098983B2
:103E3000863469F460E270E089E00E94FA1D10E2C5
:103E40000E94CD090E94DB1D1150D1F762C161E0D3
:103E500070E089E00E94FA1D52C161E070E089E0E3
:103E600053C169E170E08AE00E94FA1D82E080930C
:103E7000BA05209172058091BF059091C005A0916F
:103E8000C105B091C205222311F0806801C08F776F
:103E90008093BF059093C005A093C105B093C20560
:103EA0000AEB15E0F80181918F010E94DB1DF5E01E
:103EB000033D1F07B9F72DC161E270E08BE00E945E
:103EC000FA1D8091AA048F3F39F08091AA0491E0F5
:103ED000980F9093AA0402C08091AA040E94DB1D4F
:103EE00010E0812F0E94F7150E944C090E94E91DE5
:103EF0001F5F1031B1F70DC161E070E08CE00E94EE
:103F0000FA1D8091D30503C161E070E085E60E944F
:103F1000FA1D89E2E816F10409F0F8C0D801E6E7D5
:103F2000F5E08D91819385E0EF39F807D1F7E7C08F
:103F300061E070E086E60E94FA1DEBE1EE16F10406
:103F400009F0E4C0D801EFE9F5E08D91819385E0B7
:103F5000EA3BF807D1F7D3C061E070E087E60E9442
:103F6000FA1D0E94840DCBC061E070E088E60E94DB
:103F7000FA1D85E789838BE1EFE9F5E0DE01129612
:103F800001900D928A95E1F76CE1CE0101960E94B5
:103F90001E0C0E949C0B83E08093730560E273E02B
:103FA00080E090E00E940E2980917305843009F032
:103FB000ADC08FE70E94BA090E94CD09898385357B
:103FC00009F0A4C09CC061E070E08AE60E94FA1D7E
:103FD00089E6898361E0CE0101960E941E0C0E9451
:103FE0009C0B83E08093730560E273E080E090E0D7
:103FF0000E940E2980917305843009F087C08FE7F5
:104000000E94BA090E94CD0989838E010E5F1F4F5D
:104010007E01EDE1EE0EF11C0E94CD09F8018193C5
:104020008F01EE15FF05C1F78BE1FE013296AFE976
:10403000B5E001900D928A95E1F78981893409F004
:1040400065C05DC061E070E08BE60E94FA1DF8017A
:1040500080818093D4050E948D0D51C061E070E095
:104060008CE60E94FA1DF0E2EF16F10461F487E697
:10407000898380E2F801DE01129601900D928A9503
:10408000E1F761E203C087E4898361E0CE01019634
:104090000E941E0C0E949C0B83E0809373056CE4CD
:1040A00074E080E090E00E940E29809173058430D6
:1040B00069F58FE70E94BA090E94CD09873431F56E
:1040C0001EC061E070E08DE60E94FA1D89E1E816ED
:1040D000F104E1F4D801EAEBF5E08D91819385E0FC
:1040E000E33DF807D1F70BC061E070E08EE60E9477
:1040F000FA1DF80180818093D3050E946E0D81E046
:1041000006C061E070E08AEC0E94FA1D80E00E9427
:10411000DB1D0E94171EA196E6E00C94AC2EA0E0D9
:10412000B0E0E5E9F0E20C948E2ECAECD3E014E6A0
:1041300006E035E0F32E44E0E42E53E0D52E62E0B5
:10414000C62E82EE95E00E94EB2B892B09F49BC0D2
:1041500082EE95E00E94182C282F80933504409120
:10416000340450E04730510560F7FA01EE52FF4F3A
:104170000C94BB2E853B29F781E080933404E1CF7A
:10418000823609F07DC0C0923404DBCF80933304C3
:1041900080933204D0923404D4CF9C0133273093DF
:1041A0003104209330049091320498279093320484
:1041B000E0923404C6CF382F22274091300450912A
:1041C0003104242B352B309331042093300490910B
:1041D0003204982790933204F09234042536310546
:1041E00008F4AFCF61E070E08CEC0E94FA1D81E032
:1041F0000E94DB1D0E94171E43C020912E043091A7
:104200002F04F901E653FC4F8083909132049827E4
:1042100090933204C901019690932F0480932E0449
:1042200020913004309131048217930708F489CF2C
:104230000093340486CF8091320482130BC06091C6
:104240002E0470912F044AEC53E0809133040E94B5
:104250001E1E0DC062E070E08BEC0E94FA1D809182
:1042600033040E94DB1D80916A050E94DB1DFE0164
:10427000812F11928A95E9F710922F0410922E0443
:10428000109234045ECFCDB7DEB7E8E00C94AA2ECE
:1042900081E080936B0580916B05882349F082EE65
:1042A00095E00E94EB2B892BB1F30E948F20F3CF76
:1042B0000895AAE2B0E0EFE5F1E20C948C2E0E94A2
:1042C000DF286B017C0181E00E94C10A82EE95E04B
:1042D0000E94EB2B892B29F082EE95E00E94182C8E
:1042E000F5CF5E98409811E072E6B72EE9E2AE2E67
:1042F00003E00E94DF286C197D098E099F09693C43
:10430000710581059105E0F11123D1F10E94DF28AB
:104310006B017C015D9A419A80ED97E00E94B6079F
:10432000B982E6E7F5E0DE0112968A2D01900D9242
:104330008A95E1F76AE2CE0101960E941E0C5D9813
:10434000419880E090E00E94B607009373050E94B8
:104350009C0B62E370E080E090E00E940E29809167
:104360007305843061F4009373058FE70E94BA09E6
:104370000E94CD0911E0823419F410E001C011E06F
:1043800082E10E94042A892BA1F411E012C05E9AF6
:10439000409A5D9A419A82EE95E00E94182C8D30E9
:1043A0009105B9F06CF40A97A1F05E9840985D9879
:1043B000419882EE95E00E94EB2B892B41F799CF33
:1043C0008332910579F08234910579F70E94482172
:1043D000ECCF62EB71E082EE95E00E94C52A0E946C
:1043E000B11DE3CF0E943A16E0CF8F929F92AF9219
:1043F000BF92CF92DF92EF92FF921F93CF93DF9302
:1044000082E10E94042A892B09F089C068EC70E0DF
:1044100080E090E00E940E2980E090E00E94B607C4
:104420000E94DF284B015C016B017C0180ECC80E0F
:1044300082E1D81EE11CF11C0E94DF286C157D056D
:104440008E059F0530F482E10E94042A892BA1F396
:1044500064C082E10E94042A892B09F05EC080EDCD
:1044600097E00E94B6070E94DF286B017C01D0E034
:10447000C1E088E4880E86E2981EA11CB11C11E000
:1044800082E10E94042A892B21F58C149D04AE043C
:10449000BF0430F480ED97E00E94B607D1E0F0CF82
:1044A0000E94DF286C197D098E099F09693C7105FE
:1044B0008105910528F30E94DF286B017C01C1274B
:1044C00019F080ED97E002C080E090E00E94B6070E
:1044D000D7CF80E090E00E94B607DD23B9F080914D
:1044E000D30590E0019665E070E00E942F2E809346
:1044F000D3050E946E0D0E94EC130E948D0D64EF97
:1045000071E080E090E00E940E2909C080E00E94E6
:10451000DF060E9405120E94840D0E945921DF913E
:10452000CF911F91FF90EF90DF90CF90BF90AF9011
:104530009F908F900895CF92DF92EF92FF9280E04C
:104540000E941D080E94F40761E086E00E949829FD
:1045500061E085E00E94982961E08EE00E94982940
:1045600061E08FE00E94982960E082E10E94982932
:1045700060E088E00E94982961E088E00E94D129EB
:104580000E949F0740E052EC61E070E082EE95E00F
:104590000E94332D0E94EC130E948D0D0E94D113B6
:1045A0008FEF8093AA040E94090878940E94DF2864
:1045B0006B017C018091AA048F3F59F40E94DF288F
:1045C0006C197D098E099F09603D77408105910531
:1045D00088F380ED97E00E94B60761E082E10E94D7
:1045E000D1295E9A409A82EE95E00E94EB2B892BAE
:1045F00029F082EE95E00E94182CF5CF6DEF72E065
:1046000082EE95E00E94A62A85E893E00E94730C52
:1046100064E173E082EE95E00E94A62A4AE050E051
:1046200065E070E082EE95E00E94762B62E370E038
:1046300080E090E00E940E2982EE95E00E94EB2B34
:1046400004970CF182EE95E00E94182C82349105BB
:10465000D1F482EE95E00E94182C8E34910599F4E5
:1046600082EE95E00E94182C8434910561F482EE6C
:1046700095E00E94182C819731F480E090E00E9430
:10468000B6070E94592140917705509178056091B5
:10469000790570917A05DB01CA010197A109B10979
:1046A0000497A105B10568F44093A904433029F4A7
:1046B00040EA56E861E070E004C040E052EC61E09E
:1046C00070E082EE95E00E94332D0E94F5215E9805
:1046D000409880E090E00E94B6070E94D1131092AB
:1046E000C5048091BF0583FF11C080918B0588238D
:1046F00051F080919205882331F0809199058823AB
:1047000011F087E001C085E08093C50480E00E943D
:10471000C10A8091C6040E94F5090E949C0B109268
:104720003F0410923E0410923D04F12C8091D40578
:104730008F15B0F062E370E080E090E00E940E29F7
:1047400080ED97E00E94B60762E370E080E090E0C1
:104750000E940E2980E090E00E94B607F394E6CF15
:1047600080919E0584FF08C0982F987181E0983150
:1047700009F080E00E94C1118FE00E941D08FF90A7
:10478000EF90DF90CF900895EF92FF920F931F93D9
:10479000CF93DF938C016EE770E082EE95E00E948C
:1047A0005906E801F12CF0E2EF2E8E0188818D5739
:1047B000823048F46DE770E082EE95E00E94590681
:1047C00088818E2588832196F801608182EE95E0AC
:1047D0000E94452CF394F9E0FF12E7CF6EE770E0FA
:1047E00082EE95E00E945906CDB7DEB7E6E00C9464
:1047F000AC2EA9E0B0E0EFEFF3E20C94942E909190
:10480000C70491110EC09EEF99838A836B8350E099
:10481000559547954C832D83198618861F821E82D5
:104820002EC04091CC04842F90E0B4E095958795FC
:10483000BA95E1F7242F2F7030E08217930719F112
:104840008DEF89831B82FE01349650E0842F90E027
:10485000A4E095958795AA95E1F7242F2F7030E075
:104860008217930749F0DC01A353BB4F8C918193CE
:10487000405F5F5F563051F74093CC045A83CE01BE
:1048800001960E94C4238091C70490E0019666E0DF
:1048900070E00E942F2E8093C7042996E2E00C94CA
:1048A000B02EA0E0B0E0E7E5F4E20C948D2E6C01B0
:1048B0006EE770E082EE95E00E9459068601E12CD9
:1048C000F12CC0E0D0E030E2B32EF801608183E843
:1048D000860F823078F46DE770E082EE95E00E94FA
:1048E0005906F80160816B2570E082EE95E00E9428
:1048F000590604C082EE95E00E94452CE114F104B3
:1049000059F0F80180819E01280F311DC901C92F7E
:10491000DD27C80FD91FDD273FEFE31AF30A89E02F
:10492000E816F10459F028E0E216F10421F48C2F86
:104930008095F60180870F5F1F4FC7CFCDB7DEB7D9
:10494000E9E00C94A92EA9E0B0E0E9EAF4E20C94C5
:10495000942EE82F362F8091C70490E0019664E2F0
:1049600070E00E942F2E8093C70458E9598350E1CC
:104970005A83813089F048F08230B9F08330D9F41D
:104980008B8381EF8C833D8319C085E08B8381EF1E
:104990008C832F5F2D8312C08B8381EF8C8384E601
:1049A000489FA00111245D8309C084E08B8381EFBF
:1049B0008C83ED8303C00E94FE1104C0CE010196DA
:1049C0000E9451242996E2E00C94B02EA2E0B0E0BF
:1049D000ECEEF4E20C94892E182F762E2A8349836C
:1049E0000E94EB286B017C018091DD048090C8045B
:1049F0009090C904A090CA04B090CB042A81498148
:104A00008823C1F0D701C60188199909AA09BB09F1
:104A10004C015D0191EE89169EE29906A104B10454
:104A200020F1241708F4422F202F672D812F0E9498
:104A3000A32413C0D701C60188199909AA09BB0983
:104A40004C015D0191E3891695E79906A104B10433
:104A500060F0672D812F0E94F923C092C804D09284
:104A6000C904E092CA04F092CB042296EDE00C94C3
:104A7000A52EA2E2B0E0EFE3F5E20C948A2E8CE0E2
:104A80000E94DC0981110FC06CE173E082EE95E0B9
:104A90000E94D72A5E9A409A80E00E94C10A0E9432
:104AA0009C0B5E98409882EE95E00E94EB2B892B40
:104AB00001F182EE95E00E94182C9091A9049923AF
:104AC00019F00E94FF13EFCF40913E0450E09A018D
:104AD0002F5F3F4F2F71332760913F0470E02617FF
:104AE000370709F3FA01E75BFB4F808320933E040D
:104AF000DACF80917305843009F086C00E94EB28DC
:104B0000611571058105910549F06093B7047093B3
:104B1000B8048093B9049093BA040CC081E090E08B
:104B2000A0E0B0E08093B7049093B804A093B904D8
:104B3000B093BA048091AD049091AE0481609093DB
:104B4000AE048093AD0483E0809373058FE70E94E9
:104B5000BA0909E614E00E94CD09F80181938F019A
:104B6000F4E002371F07B9F72091720480916904BD
:104B7000982F922796FF3BC090E49227909372045F
:104B8000982F98739833F1F410E0212F30E0809142
:104B90006904877090E0821793074CF11F5F2091A2
:104BA0009E05812F90E0FC01E759FB4F24FF04C0D4
:104BB00080810E94E011E9CF608182EE95E00E9441
:104BC000452CE3CF8F7399F480916A048093B604E7
:104BD00080916B048093B40480916C048093B3043F
:104BE00080916F0490E09093AC048093AB0480912B
:104BF0003D04813019F482E080933D0480913D04AE
:104C0000833011F410923D040E94EB286B017C016B
:104C10008091AF049091B004A091B104B091B2041E
:104C20000097A105B105C9F0A7019601281B390B12
:104C30004A0B5B0BDA01C901883B9B40A105B1051A
:104C400060F00E940B0A8093B5041092AF0410929A
:104C5000B0041092B1041092B2048091BB04909100
:104C6000BC04A091BD04B091BE0446015701881A4E
:104C7000990AAA0ABB0A86E795E00E9437088616B9
:104C80009706A806B90608F4A9C0C092BB04D09242
:104C9000BC04E092BD04F092BE040E9457068091CD
:104CA000AA048830A0F08091BF059091C005A09122
:104CB000C105B091C2055CE1B695A795979587951A
:104CC0005A95D1F7892B8A2B8B2B09F0A2C18091A1
:104CD000AA048F5F8093AA048091B7049091B804CE
:104CE000A091B904B091BA040097A105B105F1F003
:104CF000C81AD90AEA0AFB0A86E795E00E94370833
:104D00006C157D058E059F0508F008C18091BF05D3
:104D100084FD04C080ED97E00E94B6071092B704AE
:104D20001092B8041092B9041092BA0490917204CF
:104D3000907C9093720450913E0480913F042091A6
:104D40003D04581709F407C1223009F004C19058F6
:104D500090937204E0919E05E770F0E0E658FC4FF6
:104D60006081693008F0DFC0615040E04613DDC06B
:104D700080933F0487E3840F90917204892B809382
:104D800072044093400483E080933D045D9A419A0D
:104D9000809183059091C50491112CC10E94BC0A99
:104DA0008091C6040E94F509E0919E05E770F0E04D
:104DB000E658FC4F608182E794E00E94D70BE091B7
:104DC000C604EF5FE093C604E83109F41FC1F0E0C8
:104DD000EA58FA4F8785882309F418C10E94460CC7
:104DE000813069F580919E05887149F18091AD040B
:104DF0009091AE04880F991F9093AE048093AD04F8
:104E000083E0809373050E949C0B0E94EB286093C3
:104E1000AF047093B0048093B1049093B204672BF5
:104E2000682B692B61F481E090E0A0E0B0E0809312
:104E3000AF049093B004A093B104B093B2048091F6
:104E40009E0584FF1FC08091AD049091AE048E7FBB
:104E50000E946D09182F6091AB048091B6040E94E6
:104E6000F513482F612F8091B50449A30E94F513D3
:104E70000091D405282F49A16091B3048091B40416
:104E80000E94E6245D9841988091C3048130C1F06E
:104E900018F08230B1F1CBC082E10E94042A892B44
:104EA00009F0C5C081E08093C3040E94DF286093AD
:104EB000BF047093C0048093C1049093C204B7C030
:104EC00082E10E94042A892B31F50E94DF28C090DC
:104ED000BF04D090C004E090C104F090C2046C19EB
:104EE0007D098E099F09693E73408105910508F48B
:104EF0009EC082E08093C30480ED97E00E94B607D5
:104F000096C082E10E94042A892B09F490C080E0B7
:104F100090E00E94B6071092C30489C080E090E040
:104F20000E94B60703CF68E020CF851709F420CF91
:104F30004F5F242F30E090E0F901EE58FB4FDC0189
:104F4000A75BBB4F7C917083F901E05CFB4F7083E2
:104F500001968F710BCF2430B1F42091400481E48D
:104F600094E0A3E7B4E0FC013E2F381B321718F49D
:104F700031913D93F9CF87E3820F90917204892B91
:104F80008093720400CF8091C304823059F4916001
:104F9000909372045E9A409A8E010F5F1F4FF12C1E
:104FA000B80111C05E98409880913D04811103C002
:104FB00081E080933D0480913D04833069F784E073
:104FC00080933D04E9CF8F2D69A37AA30E94F71542
:104FD000F801819391938F01F39469A17AA1F0E193
:104FE000FF12F1CF80919E0543E754E087700E9445
:104FF000BC08CCCE882309F4D1CE2091C40431E082
:10500000320F3093C4042913C9CE0DC01092C604C8
:10501000E5CE8091AA04883011F45E9A409A89E026
:105020008093AA04DBCE1092C4048150B7CEA2961E
:10503000ECE00C94A62E8230E8F4E82FF0E0EE0FBE
:10504000FF1FEB52FA4F71836083813041F08091F2
:1050500069008C7F842B80936900E89A0895809181
:105060006900440F551F440F551F837F842B809385
:105070006900E99A08951F920F920FB60F921124BA
:105080002F933F934F935F936F937F938F939F9350
:10509000AF93BF93EF93FF938091D5059091D60581
:1050A000892B29F0E091D505F091D6050995FF915E
:1050B000EF91BF91AF919F918F917F916F915F9190
:1050C0004F913F912F910F900FBE0F901F90189509
:1050D0001F920F920FB60F9211242F933F934F936D
:1050E0005F936F937F938F939F93AF93BF93EF9350
:1050F000FF938091D7059091D805892B29F0E091F5
:10510000D705F091D8050995FF91EF91BF91AF9127
:105110009F918F917F916F915F914F913F912F91CF
:105120000F900FBE0F901F9018951F920F920FB601
:105130000F9211242F933F938F939F93AF93BF931D
:105140008091DA059091DB05A091DC05B091DD0539
:105150003091D90523E0230F2D3720F40196A11DAE
:10516000B11D05C026E8230F0296A11DB11D209395
:10517000D9058093DA059093DB05A093DC05B09305
:10518000DD058091DE059091DF05A091E005B091ED
:10519000E1050196A11DB11D8093DE059093DF0509
:1051A000A093E005B093E105BF91AF919F918F91DE
:1051B0003F912F910F900FBE0F901F9018952FB712
:1051C000F8946091DA057091DB058091DC0590918F
:1051D000DD052FBF08953FB7F8948091DE059091CB
:1051E000DF05A091E005B091E10526B5A89B05C0BB
:1051F0002F3F19F00196A11DB11D3FBF6627782FE3
:10520000892F9A2F620F711D811D911D42E0660F3B
:10521000771F881F991F4A95D1F70895CF92DF9283
:10522000EF92FF92CF93DF936B017C010E94EB28FA
:10523000EB01C114D104E104F10479F00E94EB28E0
:105240006C1B7D0B683E7340A0F381E0C81AD10847
:10525000E108F108C851DC4FECCFDF91CF91FF900E
:10526000EF90DF90CF900895789484B5826084BDEC
:1052700084B5816084BD85B5826085BD85B581605A
:1052800085BDEEE6F0E0808181608083E1E8F0E0BA
:105290001082808182608083808181608083E0E8E9
:1052A000F0E0808181608083E1EBF0E080818460C8
:1052B0008083E0EBF0E0808181608083EAE7F0E0CA
:1052C000808184608083808182608083808181602E
:1052D00080838081806880831092C100089583302C
:1052E00081F028F4813099F08230A1F00895863061
:1052F000A9F08730B9F08430D1F4809180008F7D9F
:1053000003C0809180008F7780938000089584B5DA
:105310008F7702C084B58F7D84BD08958091B000E1
:105320008F7703C08091B0008F7D8093B000089587
:10533000CF93DF9390E0FC01ED50F44F2491FC01FA
:10534000E95FF34F8491882349F190E0880F991F1A
:10535000FC01E15DF34FA591B4918B5D934FFC018E
:10536000C591D4919FB7611108C0F8948C91209594
:1053700082238C93888182230AC0623051F4F8948E
:105380008C91322F309583238C938881822B888354
:1053900004C0F8948C91822B8C939FBFDF91CF91A6
:1053A0000895A1E0B0E0E7EDF9E20C94922E282FE9
:1053B00030E0F901E152F44F8491F901ED50F44FDE
:1053C0001491F901E95FF34F04910023C9F0882398
:1053D00021F069830E946F296981E02FF0E0EE0FD0
:1053E000FF1FEB5DF34FA591B4919FB7F8948C919B
:1053F000611103C01095812301C0812B8C939FBF45
:105400002196E4E00C94AE2ECF93DF93282F30E06A
:10541000F901E152F44F8491F901ED50F44FD49128
:10542000F901E95FF34FC491CC2391F081110E94FF
:105430006F29EC2FF0E0EE0FFF1FE55EF34FA59113
:10544000B4912C912D2381E090E021F480E002C002
:1054500080E090E0DF91CF9108958E3008F08E507B
:10546000877020919D0190E4299F90011124822B47
:1054700080937C0080917A00806480937A00809190
:105480007A0086FDFCCF809178002091790090E031
:10549000922B0895A0E0B0E0E0E5FAE20C948E2EA5
:1054A0006C017A01EB01E60EF71E00E010E0CE156C
:1054B000DF0561F06991D601ED91FC910190F081D9
:1054C000E02DC6010995080F191FF1CFC801CDB70E
:1054D000DEB7E8E00C94AA2E6115710589F0DB01B6
:1054E0000D900020E9F7AD0141505109461B570BC3
:1054F000DC01ED91FC910280F381E02D0995089586
:1055000080E090E00895EF92FF920F931F93CF9366
:10551000DF938C01FB01C0E0D0E064917F018FEF4D
:10552000E81AF80A662361F0D801ED91FC91019028
:10553000F081E02DC8010995C80FD91FF701EDCF03
:10554000CE01CDB7DEB7E6E00C94AC2E0E946C2AFB
:105550000895DC01ED91FC910190F081E02D099519
:1055600008950F931F93CF93DF93EC016DE00E949A
:10557000A92A8C016AE0CE010E94A92A800F911FFE
:10558000DF91CF911F910F9108950F931F93CF93A8
:10559000DF93EC010E94832A8C01CE010E94B12A84
:1055A000800F911FDF91CF911F910F9108950F935D
:1055B0001F93CF93DF93EC010E946C2A8C01CE01E4
:1055C0000E94B12A800F911FDF91CF911F910F91FF
:1055D00008950F931F93CF93DF93EC010E94A92AA4
:1055E0008C01CE010E94B12A800F911FDF91CF91D3
:1055F0001F910F910895A1E2B0E0E1E0FBE20C946D
:105600008A2E7C01C42EE52FCB01D22E19A221E0D7
:105610002D1510F02AE0D22E8E010F5D1F4F8D2C1C
:10562000912CA12CB12C6C2D7E2FA50194010E94F0
:10563000432E8C2DD29E80191124015011098A30DD
:1056400010F4805D01C0895CF8018083211531056B
:105650004105510521F0C22EE32FCA01E4CFB80164
:10566000C7010E946C2AA196ECE00C94A62EA0E043
:10567000B0E0EDE3FBE20C948E2EEC016A017B01BD
:105680002115310541F4E881F9810190F081E02D87
:10569000642F09951DC02A303105A9F477FF12C087
:1056A0006DE20E94A92A8C0144275527BA014C19A2
:1056B0005D096E097F092AE0CE010E94FB2A800F56
:1056C000911F06C02AE0B701A601CE010E94FB2A65
:1056D000CDB7DEB7E8E00C94AA2E9A01AB0166279D
:1056E00057FD6095762F0E94372B08950F931F93D7
:1056F000CF93DF93EC019A01AB01662757FD6095CC
:10570000762F0E94372B8C01CE010E94B12A800F88
:10571000911FDF91CF911F910F91089521153105B0
:1057200049F4DC01ED91FC910190F081E02D642FB2
:10573000099508950E94FB2A08959A01462F50E08A
:1057400060E070E00E948E2B08959A01AB0160E04A
:1057500070E00E948E2B08950F931F93CF93DF93D9
:10576000EC010E948E2B8C01CE010E94B12A800F89
:10577000911FDF91CF911F910F9108950F931F9368
:10578000CF93DF93EC019A01AB0160E070E00E94DF
:105790008E2B8C01CE010E94B12A800F911FDF91C8
:1057A000CF911F910F9108950F931F93CF93DF9384
:1057B000EC019A01462F50E060E070E00E948E2BD1
:1057C0008C01CE010E94B12A800F911FDF91CF91F1
:1057D0001F910F910895FC0124853585F901E05C46
:1057E000FF4F80819181F901EE5BFF4F2081318174
:1057F000821B930B8F7399270895FC0184859585EF
:10580000FC01E05CFF4F40815181FC01EE5BFF4FEA
:10581000208131814217530741F00190F081E02D42
:10582000E80FF91F808190E008958FEF9FEF0895B2
:10583000FC0184859585FC01E05CFF4F408151812E
:10584000FC01EE5BFF4F208131814217530779F055
:10585000A081B181A80FB91F8C91208131812F5F68
:105860003F4F2F7333273183208390E008958FEFCC
:105870009FEF0895FC0181A1882329F0A489B589AF
:105880008C9186FFFBCF11A20895CF93DF93FC018B
:1058900026853785D901A05CBF4F8D919C911197CA
:1058A00001968F739927E901CE5BDF4F48815981BB
:1058B00084179507D9F30D90BC91A02DA20FB31FAB
:1058C0006C93A685B785A05CBF4F11969C938E9371
:1058D000A689B7892C9181E090E0078C02C0880FDF
:1058E000991F0A94E2F7282B2C9381E081A3048866
:1058F000F589E02D80818064808381E090E0DF91F4
:10590000CF91089508951F920F920FB60F92112410
:105910002F933F934F938F939F93EF93FF93809198
:10592000C00082FD1CC04091C60080918806909105
:10593000890601968F73992720918A0630918B06EC
:105940008217930771F0E0918806F0918906E85B71
:10595000F94F4083909389068093880602C0809116
:10596000C600FF91EF919F918F914F913F912F91A1
:105970000F900FBE0F901F90189582EE95E00E9439
:10598000EB2B892B11F00E94822C08951F920F920D
:105990000FB60F9211242F933F938F939F93EF9302
:1059A000FF932091440630914506809146069091E0
:1059B00047062817390731F48091C1008F7D809305
:1059C000C10014C0E0914606F0914706EC5FF94F24
:1059D0002081809146069091470601968F73992702
:1059E00090934706809346062093C600FF91EF915F
:1059F0009F918F913F912F910F900FBE0F901F900D
:105A00001895A0E0B0E0E7E0FDE20C948A2EFC01DE
:105A10001382128288EE93E0A0E0B0E08483958345
:105A2000A683B7838CEB93E091838083758764872B
:105A300057874687318B208B138B028BF58AE48A3C
:105A4000D78AC68AB18EA08E938E828E8F85848FE0
:105A50008889858F8989868F8A89878F8B8980A39A
:105A6000ECE00C94A62ECF92DF92EF92FF92CF93B0
:105A7000DF93EC016A017B01411581EE5807610556
:105A80007105F9F0EC89FD8981E090E008A002C081
:105A9000880F991F0A94E2F7808360E079E08DE334
:105AA00090E0A70196010E94432E2150310941093F
:105AB00051095695479537952795211580E1380767
:105AC00098F0EC89FD89108260E874E88EE190E03E
:105AD000A70196010E94432E215031094109510925
:105AE0005695479537952795E889F9893083EA894E
:105AF000FB89208319A2EE89FF89408181E090E033
:105B00009C010C8C02C0220F331F0A94E2F7422B37
:105B10004083EE89FF8940819C010D8C02C0220FD9
:105B2000331F0A94E2F7422B4083EE89FF894081BC
:105B30009C010E8C02C0220F331F0A94E2F7422B05
:105B40004083EE89FF8920810F8C02C0880F991F46
:105B50000A94E2F7809582238083DF91CF91FF90B2
:105B6000EF90DF90CF9008958F929F92AF92BF9267
:105B7000CF92DF92EF92FF920F931F9381E08F936A
:105B800085E08F9387E08F9383E08F9384E08F93FA
:105B9000E6EC8E2E912CF2ECAF2EB12CA1ECCA2E9D
:105BA000D12CB0ECEB2EF12C04EC10E025EC30E025
:105BB00044E056E068E476E082EE95E00E94012D34
:105BC0000F900F900F900F900F901F910F91FF90DB
:105BD000EF90DF90CF90BF90AF909F908F900895FF
:105BE0000E9434290E949B22CDEBDCE20E943925E1
:105BF0002097E1F30E94BD2CF9CFA29FB001B39F83
:105C0000C001A39F700D811D1124911DB29F700DC5
:105C1000811D1124911D08950E94FD2DA59F900DB9
:105C2000B49F900DA49F800D911D11240895B7FF7E
:105C30000C940C2E0E940C2E821B930B0895DB01FA
:105C40008F939F930E940C2EBF91AF91A29F800DC6
:105C5000911DA39F900DB29F900D1124089597FB65
:105C6000072E16F4009407D077FD09D00E94C12EAC
:105C700007FC05D03EF4909581959F4F089570954F
:105C800061957F4F0895A1E21A2EAA1BBB1BFD014F
:105C90000DC0AA1FBB1FEE1FFF1FA217B307E4070B
:105CA000F50720F0A21BB30BE40BF50B661F771F63
:105CB000881F991F1A9469F7609570958095909543
:105CC0009B01AC01BD01CF010895052E97FB1EF489
:105CD00000940E947C2E57FD07D00E94432E07FCA3
:105CE00003D04EF40C947C2E509540953095219520
:105CF0003F4F4F4F5F4F08959095809570956195F8
:105D00007F4F8F4F9F4F08952F923F924F925F92F8
:105D10006F927F928F929F92AF92BF92CF92DF92BB
:105D2000EF92FF920F931F93CF93DF93CDB7DEB720
:105D3000CA1BDB0B0FB6F894DEBF0FBECDBF0994B4
:105D40002A88398848885F846E847D848C849B840B
:105D5000AA84B984C884DF80EE80FD800C811B8119
:105D6000AA81B981CE0FD11D0FB6F894DEBF0FBE48
:105D7000CDBFED010895EE0FFF1F0590F491E02DCA
:105D80000994AA1BBB1B51E107C0AA1FBB1FA61782
:105D9000B70710F0A61BB70B881F991F5A95A9F7D4
:105DA00080959095BC01CD0108958F929F92AF92FE
:105DB000BF92CF92DF92EF92FF92CF93DF93EC01ED
:105DC000688179818A819B816115710581059105C1
:105DD00021F464E279ED8BE597E02DE133EF41E0CA
:105DE00050E00E94652E49015A019B01AC01A7EACF
:105DF000B1E40E940C2E6B017C01ACEEB4EFA50166
:105E000094010E941A2EC60ED71EE81EF91EF7FE38
:105E100006C081E0C81AD108E10880E8F80AC88203
:105E2000D982EA82FB82C701B6019F77DF91CF91C9
:105E3000FF90EF90DF90CF90BF90AF909F908F90AA
:105E400008950E94D52E089586E091E00E94D52EF7
:105E50000895609306017093070180930801909361
:105E6000090108952F923F925F926F927F928F92D5
:105E70009F92AF92BF92CF92DF92EF92FF920F93D9
:105E80001F93CF93DF938B01EA016115710521F018
:105E9000DB018C9311969C93209739F09E01225040
:105EA00031092332310508F0D8C07C016701BFEF0A
:105EB000CB1ADB0A5601F7016080862D90E00E9424
:105EC0006430892B11F07601F1CFFDE26F120AC028
:105ED000570182E0A80EB11CD70111966C9077246F
:105EE00073940BC0BBE26B1207C05701E2E0AE0E29
:105EF000B11CD70111966C90712CCE018F7E892B2D
:105F000089F4B0E36B1237C0F50180818F7D88354D
:105F1000D1F46180F2E0AF0EB11C872D8260782E43
:105F2000C0E1D0E0CA30D10551F1C031D10521F036
:105F3000C830D10599F409C0CC24CA94DC2CEC2CCF
:105F4000AFE0FA2E22C0209769F7C8E0D0E0CC2459
:105F5000CA94DC2CEC2CFFE1FF2E17C06FEF7FEF13
:105F6000CB019E01442737FD4095542F0E94432EBC
:105F700069017A010AC02097A9F6CAE0D0E0E9E9F0
:105F8000CE2EDC2CEC2CE9E1FE2EF50160E020E0C9
:105F900030E0A9014E01AA2497FCA094BA2C1F015D
:105FA00070ED572E560CA9E0A51570F48FEB860DF9
:105FB0008A3118F499EC592E06C08FE9860D8A3182
:105FC00048F589EA582E560C852D90E08C179D07D0
:105FD0000CF56F3FD9F0C216D306E406F50698F02B
:105FE000C501B4010E941F2E9B01AC01852D90E0DC
:105FF000A0E0B0E0280F391F4A1F5B1F28173907A0
:106000004A075B0710F46FEF01C061E03196D101E0
:106010006C90C5CF0115110551F0662311F0319731
:1060200003C071FE04C03297D801ED93FC9370FE5B
:1060300007C050954095309521953F4F4F4F5F4F8A
:1060400067FF10C082E290E090938D0680938C06EB
:106050006FEF7FEF8FEF9FEF07C060E070E080E0B1
:1060600090E002C0B901CA01DF91CF911F910F9159
:10607000FF90EF90DF90CF90BF90AF909F908F9068
:106080007F906F905F903F902F900895FC0188273C
:106090009927E89421912032E9F3293010F02E302D
:1060A000C8F32B3241F02D3239F4689404C00E94B9
:1060B0009830820F911D219120532A30C0F31EF495
:1060C000909581959F4F0895911150C0803219F09D
:1060D00089508550D0F7089548EC53E00E94713004
:1060E0000895FA01A191B081009719F41097E1F099
:1060F000CD01DC01CD010D90002011F4C00113C0D1
:10610000FB012191222319F02015D9F7F3CFFB01D0
:106110002191201519F41E92119606C02223C1F771
:106120000D900020A1F7D001FA01A193B08308954A
:106130007AE0979F902D879F802D910D11240895CF
:10614000F999FECF92BD81BDF89A992780B508953F
:10615000262FF999FECF1FBA92BD81BD20BD0FB683
:10616000F894FA9AF99A0FBE01960895992788270C
:066170000895F894FFCF32
:1061760000008E06200001000000FF000200020061
:1061860002000200020002000200020002000200F9
:106196000200020002000200020002802500000543
:1061A600400AA1204EA50020244EA52C2330C01263
:1061B60000001A400AA1204EA5001B1E27522C23C0
:1061C600308025000005400AA1204EA50020244E5F
:1061D600A52C2330004B000006400AD0009D490044
:1061E6007B289D492C233000E1000005400A45012B
:1061F600D7DC03B81E0EBF00232E48E801008A40F4
:106206000A6001555502AD1E20000023C8015458EE
:106216002074696D656F75742100596573004E6F42
:10622600002C00386368004E2F41002C205B005D77
:106236002028002900486F70206368616E6E656CC7
:10624600200020402000456E746572696E672061EB
:1062560064617074697665206368616E6E656C2032
:1062660073656C656374696F6E2C207069636B6906
:106276006E673A007363616E6E6572206D6F64655A
:10628600004E4F5420454E41424C45440053656EE6
:1062960064696E672073657474696E677320746FC2
:1062A6002052580A00526573657474696E672073CC
:1062B600657474696E6773206F6E2052580A0041C8
:1062C600626F727465642065646974730A00696E2E
:1062D60076616C69642073656C656374696F6E00C2
:1062E6000D0A496E76616C696420696E707574205A
:1062F6002D206469736361726465642107005365C8
:106306007474696E677320736176656420746F2098
:10631600454550524F4D0A00526576657274656464
:106326002073657474696E67732066726F6D20459D
:106336004550524F4D0A004C6F616465642066619A
:1063460063746F72792064656661756C74730A0094
:106356004B657920616E64206368616E6E656C734F
:106366002072616E646F6D697A65640A004F7065AC
:106376006E4C52536E672054582073746172746960
:106386006E672000206F6E20485720006D6F647581
:106396006C65206C6F636B65643F00342B3400388A
:1063A60000382B340031320031322B3400313600C4
:1063B60050504D0052535349005344410053434CEF
:1063C60000525844005458440041494E004C42453E
:1063D60045500053504B54524D00534255530053B1
:1063E600554D44004C4C494E440000070B0C10110F
:1063F6001500B7012B032F033103350338033D0383
:10640600B7014003440349034D03510355035903A0
:106416005D0363036A036F0374038D028D028D02AD
:106426008D02160A1322312900000000452C4A2A43
:08643600EB2B182CFD2B3A2C76
:107E00000F92CDB7DEB7112484B714BE81FFF1D035
:107E100082E08093C00088E18093C10086E0809377
:107E2000C20080E18093C4008EE0CDD088249924E4
:107E3000CC24C394F5E0DF2EE1E1EE2E73E0F72EC3
:107E4000B6D0082F813479F4B2D08983C2D0898129
:107E5000823811F481E005C0813811F485E001C059
:107E600083E09ED09AC0823411F484E103C085344B
:107E700019F485E0B6D091C0853561F498D0082F0B
:107E800010E095D090E0982E8824802A912A880CC2
:107E9000991C82C0863521F484E0A3D080E0E1CF34
:107EA000843609F04CC083D082D0A82E80D0B82E62
:107EB00000E011E07CD0F80181938F01AE16D1F77C
:107EC00088D0FB2DF53489F4E0E0F1E00BC0F9999E
:107ED000FECF92BC81BC0894811C911C819180BD15
:107EE000FA9AF99AEA1598F358C08B2D863409F05E
:107EF00054C0F401F7BEE89507B600FCFDCFF401CD
:107F0000A0E0B1E02C9130E011968C91119790E0B7
:107F1000982F8827822B932B12960C01C7BEE895C9
:107F20001124329681E0A038B80761F7F401D7BE7A
:107F3000E89507B600FCFDCFE7BEE8952EC0843774
:107F4000F1F435D034D0182F32D0B82E42D0FB2DDA
:107F5000F63421F4F40105914F010CC0FB2DF534EA
:107F600049F4F999FECF92BC81BC0894811C911C04
:107F7000F89A00B5802F14D0115049F70EC08537FC
:107F800039F427D08EE10CD085E90AD08FE069CF93
:107F9000813511F488E017D01CD080E101D050CF9A
:107FA0009091C00095FFFCCF8093C600089580910A
:107FB000C00087FFFCCF8091C00084FD01C0A89560
:107FC0008091C6000895E0E6F0E098E19083808318
:107FD0000895EDDF803219F088E0F5DFFFCF84E10E
:107FE000DFCF1F93182FE3DF1150E9F7F2DF1F9166
:0E7FF0000895282E80E0E7DFEE27FF27099492
:027FFE0001057B
:0400000300007E007B
:00000001FF
